:0200000480007A
:100000009710000093800000171100001301810277
:1000100083A1000013020000930210001303F0FFFD
:10002000B70300809383F3FF37040080338241409D
:10003000B382514033836140B38371403384814044
:100040002320310023224100232451002326610074
:1000500023287100232A8100971000009380C0FAA2
:1000600017110000130181FE03A400009304000097
:10007000130510009305F0FF370600801306F6FF06
:10008000B7060080B30494403305A440B305B440E0
:100090003306C440B306D4402320810023229100BC
:1000A0002324A1002326B1002328C100232AD10044
:1000B00097100000938080F517110000130181FA5A
:1000C00083A6000013070000930710001308F0FF39
:1000D000B70800809388F8FF370900803387E6402F
:1000E000B387F64033880641B388164133892641E9
:1000F0002320D1002322E1002324F1002326010143
:1001000023281101232A210197100000938040F039
:1001100017110000130181F603A9000093090000E4
:10012000130A1000930AF0FF370B0080130BFBFF3C
:10013000B70B0080B3093941330A4941B30A594129
:10014000330B6941B30B7941232021012322310173
:10015000232441012326510123286101232A71010F
:1001600097100000938000EB17110000130181F23B
:1001700083AB0000130C0000930C1000130DF0FF74
:10018000B70D0080938DFDFF370E0080338C8B41BF
:10019000B38C9B41338DAB41B38DBB41338ECB418F
:1001A0002320710123228101232491012326A1010F
:1001B0002328B101232AC101971C0000938CCCE5B0
:1001C000171D0000130D8DEE03AE0C00930D1000F3
:1001D000B30EBE41338FBE41B30FBF41B380BF41A9
:1001E0003381B041B301B1412320BD012322CD01B0
:1001F0002324DD012326ED012328FD01232A1D00F0
:10020000232C2D00232E3D0097100000938000E149
:1002100017110000130181EB03AE0000B79DFFF73B
:10022000938D8D813300BE41232001009710000083
:10023000938000DF17110000130181E903AE000075
:10024000B79DFFF7938D8D813300BE41B30200400F
:10025000232001002322510097100000938080DCAE
:1002600017110000130141E783A100003382014010
:10027000B30202403303504033070340B307074043
:1002800033880740B30C0041330D9041B30D0D404E
:10029000232041002322A1012324B10117150000CE
:1002A000130545D9971500009385C5E3370610F06F
:1002B0001306C6F26306B5028326C5002320D600C6
:1002C000832685002320D600832645002320D600E0
:1002D000832605002320D600130505016FF09FFD3E
:1002E000370510F0130505F223200500000000007B
:0402F000000000000A
:101000000000000001000000FFFFFFFFFFFFFF7F67
:1010100000000080CDAB00007856341298BADCFE98
:10102000145892360000000000000000000000008C
:10103000FFFFFFFFFFFFFFFFFFFFFFFFFFFFFFFFC0
:10104000FFFFFFFFFFFFFFFFFFFFFFFFFFFFFFFFB0
:10105000FFFFFFFFFFFFFFFFFFFFFFFFFFFFFFFFA0
:10106000FFFFFFFFFFFFFFFFFFFFFFFFFFFFFFFF90
:10107000FFFFFFFFFFFFFFFFFFFFFFFFFFFFFFFF80
:10108000FFFFFFFFFFFFFFFFFFFFFFFFFFFFFFFF70
:10109000FFFFFFFFFFFFFFFFFFFFFFFFFFFFFFFF60
:1010A000FFFFFFFFFFFFFFFFFFFFFFFFFFFFFFFF50
:1010B000FFFFFFFFFFFFFFFFFFFFFFFFFFFFFFFF40
:1010C000FFFFFFFFFFFFFFFFFFFFFFFFFFFFFFFF30
:1010D000FFFFFFFFFFFFFFFFFFFFFFFFFFFFFFFF20
:040000058000000077
:00000001FF
